:1000000013C01AC019C018C017C016C015C014C03C
:1000100013C012C011C010C00FC00EC00DC03F06EB
:100020005B4F666D7D077F6F11241FBECFE5D1E06A
:10003000DEBFCDBF30D11EC3E3CFF894C09AC29AC1
:100040008DE08A95F1F70000C0988DE08A95F1F770
:100050000000C29878940895F894C298C0988DE0F2
:100060008A95F1F70000C29A8DE08A95F1F70000B9
:10007000C09A78940895F8942DE02A95F1F700003D
:1000800098E00DC0C09886952DE02A95F1F7000004
:10009000C29A2DE02A95F1F70000915049F0C298DC
:1000A0002DE02A95F1F7000080FFECCFC09AEBCF4E
:1000B000B898C298C09A8DE08A95F1F7000086B38F
:1000C000C29A9DE09A95F1F70000C2982DE02A951A
:1000D000F1F70000B89A7894809581700895CF93D5
:1000E000C82FABDF8C2FC7DFB7DFCF91089597B351
:1000F000A1E0B0E0FD0102C0EE0FFF1F8A95E2F71C
:1001000002C0AA0FBB1F6A95E2F7EA2B9E2B97BB92
:1001100088B3E095E823E8BB842F8068822BDFDF7B
:100120000895CF93DF93C82FD62F80E4D8DF85DFE3
:100130008D2F806CA0DF8C2F9EDF8EDFDF91CF9123
:10014000089562E080E4EDDF61E080E4EADF60E0F2
:1001500080E4E7DF089521E08A30910550F021E046
:10016000EAE0F0E0BF015FD2CB012F5F6A3071059A
:10017000C8F7822F0895AF92BF92CF92DF92EF928D
:10018000FF920F931F93CF93DF9300D01F92CDB7B1
:10019000DEB7B62EF42E009749F461113BC08C01F6
:1001A000883E93407CF007EE13E00CC08C01883E43
:1001B00023E0920714F007EE13E099231CF4119545
:1001C00001951109C801C7DFA82E2AE030E0C80157
:1001D000B9013DD28B83CB01B90139D28A83C801E1
:1001E00064E670E034D2CB01B90131D2898331E0C9
:1001F000A31691F083E0D82EDA1882E08D15A8F1CD
:1002000010E000E0C12C82E090E09C012F19310940
:10021000790118C08C01D3CFDA2CF2CFE1E0F0E005
:10022000EC0FFD1FED0DF11DE081F0E0E25EFF4FF0
:1002300084916C2D76DFD394C3940F5F1F4F82E0BF
:100240008D15A0F0E016F10649F733E0A31631F35F
:10025000E1E0F0E0EC0FFD1FED0DF11DE081F0E0BD
:10026000E25EFF4F84918068E4CFC12CEB2DF0E07B
:10027000E25EFF4F84916C2D54DF0F900F900F9032
:10028000DF91CF911F910F91FF90EF90DF90CF9072
:10029000BF90AF900895CF93DF93CDB7DEB764974B
:1002A0000FB6F894DEBF0FBECDBF6BE0CE01019656
:1002B000E5D028E042E062E080E019DF42DF04E6BA
:1002C00010E001C03EDFCE01019613D18111FACFBB
:1002D000CE01019621D18B899C89B801A4D141E03E
:1002E00089899A8948DFEFCFF894BC9A8FEB93E025
:1002F0000197F1F700C00000BC989AEB9A95F1F7CE
:1003000000C086B3E3E3F3E03197F1F700C00000EB
:1003100078948295817091E08927089598E00DC0C6
:10032000BC9A20EA2A95F1F7BC982AE12A95F1F7C0
:1003300000C078948695915069F0F89480FFF0CFD2
:10034000BC9A20E12A95F1F7BC982AEA2A95F1F7A0
:1003500000C0EFCF089598E080E007C022E92A9519
:10036000F1F700C07894915071F0F8948695BC9A9A
:1003700020E12A95F1F7BC9828E12A95F1F7B49B82
:10038000EDCF8068EBCF0895AFDF811101C00895F4
:100390008CECC4DF81E0FBCF0F931F93CF93DF93EF
:1003A0008C01A2DF811105C0DF91CF911F910F91C8
:1003B000089583E3B3DFE801085F1F4FCCDF899323
:1003C000C017D107D9F781E0EFCFFC01680F791F83
:1003D00080E02CE80BC08695915029F080FFFBCF80
:1003E00086958227F9CFE617F70721F091918927A3
:1003F00098E0F4CF0895EF92FF920F931F93CF935D
:10040000DF937C01C1DF8EEB89DFE7018701085FA5
:100410001F4FA1DF8993C017D107D9F768E070E0BB
:10042000C701D3DFC82F97DF91E0C81390E0892F71
:10043000DF91CF911F910F91FF90EF90089554DFBE
:10044000811101C00895A0DF88E468DF8FE19EE498
:100450000197F1F700C0000081E0F4CFCF93DF9364
:10046000EC0192DF8EE45ADF888158DF898156DF04
:100470008A8154DFE4DFDF91CF910895FF920F93DB
:100480001F93CF93DF9300D01F92CDB7DEB78C01BF
:10049000F62EB1DFF8018281898383818A83FAE0B5
:1004A000FF16B9F08BE0F81689F0E9E0FE16A1F02E
:1004B0008FE78B83CE010196D1DF0F900F900F90C5
:1004C000DF91CF911F910F91FF9008958FE58B835E
:1004D000F1CF8FE38B83EECF8FE18B83EBCF04DF04
:1004E000811101C008958CEC19DF84E417DF81E0ED
:1004F000F9CFCF93DF93EC01F7DE811104C081E0E7
:10050000DF91CF910895CE01089646DF81E098856E
:100510009832B1F780E0F4CFCF93DF93EC01DFDFC7
:10052000882309F456C02C81822F90E08095909505
:1005300080769927892B09F04FC02FE78FE492E14D
:10054000215080409040E1F700C00000CE0153DF11
:10055000882309F43EC029813881522F432FCA01D4
:1005600099230CF45BC095958795959587959595FE
:10057000879595958795998B888B287F11F0319574
:10058000388388818F70282F30E0C901880F991F28
:1005900082959295907F9827807F9827821B930B56
:1005A000880F991F880F991F820F931F880F991F1B
:1005B000880F991F880F991F9C0199238CF13595FD
:1005C00027953595279535952795359527953B8B17
:1005D0002A8BDF91CF91089526FF0AC02FEB87E287
:1005E00099E0215080409040E1F700C00000AECF7C
:1005F00025FF0AC02FEF86E994E02150804090400B
:10060000E1F700C00000A2CF2FE78BE492E0215079
:1006100080409040E1F700C0000098CF0F96A3CF34
:10062000215F3F4FCCCFAA1BBB1B51E107C0AA1FC4
:10063000BB1FA617B70710F0A61BB70B881F991F83
:100640005A95A9F780959095BC01CD01089597FB27
:10065000072E16F4009406D077FD08D0E4DF07FCDF
:1006600005D03EF4909581959F4F089570956195C2
:080670007F4F0895F894FFCFBD
:00000001FF
